:020000040000FA
:02000000802856
:080008008312692069208101C7
:100010000B11A00A0F302002031D54288312860AF8
:10002000A001A10AC730E120303021076E20ED2069
:100030000A302102031D5428A101A20AC630E12082
:10004000303022077720ED2006302202031D54288D
:10005000A201A30AC430E120303023076E20ED2036
:100060000A302302031D5428A301A40AC330E1204F
:10007000303024077720ED2006302402031D542859
:10008000A401A50AC130E120303025076E20ED2003
:100090000A302502031D5428A501A60AC030E1201C
:1000A00030302607ED2054288B160900A001A1014D
:1000B000A201A301A401A501A601080004302502A4
:1000C000031DA12802302602031DA1285620B020BE
:1000D0000800BB30A800A80B6B280800A7003A3026
:1000E0002702031D75283030080027080800A700E4
:1000F00036302702031D7E2830300800270808000C
:1001000007309F0083169F01003086008500831210
:100110003830E1200130E1200330E1200F30E120D0
:100120008030E120C030E120A320B02007308316CA
:100130008100831205108601003081008B178B1619
:1001400086015E20A1280030A1000030A20000300E
:10015000A3000230A4000530A5000130A60008006D
:10016000C730E12030302107ED20C630E1203030AB
:100170002207ED20C530E1203A30ED20C430E120E7
:1001800030302307ED20C330E12030302407ED204C
:10019000C230E1203A30ED20C130E1203030250777
:1001A000ED20C030E12030302607ED208030E12006
:1001B0005430ED204930ED204D30ED204530ED201C
:1001C00008008600F92004308500F9200030850001
:1001D000F92004308500F92008008600F920063057
:1001E0008500F92002308500F92006308500F920CD
:1001F00008001930AA00A900A90BFC28AA0BFB28AB
:100200000800FA30AA00A900A90B0429AA0B0329A7
:08021000080001210121012178
:02400E00293F48
:00000001FF
